:100000000828FF3FFF3FFF3F742E332D8A018200F7
:10001000FF30A200FF30A3005A250A30CD2525125B
:100020002926033051253230ED2503305125323059
:10003000ED25033051253230ED253230452528306D
:1000400045251325F7241125850107309F00231727
:100050004726A3164826A317462622114B268501BC
:1000600007309F00AB01AC01A0102325B701013080
:10007000B60023240130CA001E264B08B00002300F
:10008000CA001E264B08AE000330CA001E264B08CD
:10009000B1002E086C3C031CB2280430CA001E2696
:1000A0004B08B3000530CA001E264B08B2000630CC
:1000B000CA001E264B08A8000730CA001E264B089F
:1000C000A9000830CA001E264B08B8000930CA0033
:1000D0001E264B08B9000A30CA001E264B08BA007B
:1000E0000B30CA001E264B08BB000C30CA001E266F
:1000F0004B08BC000D30CA001E264B08BD000E3058
:10010000CA001E264B08BE000F30CA001E264B0830
:10011000BF001030CA001E264B08C0001130CA00B4
:100120001E264B08C1001230CA001E264B08C20012
:100130001330CA001E264B08C3001430CA001E2606
:100140004B08C4001530CA001E264B08C5001630E7
:10015000CA001E264B08C6001730CA001E264B08D0
:10016000C700B6280B30B2004630B3000230CD25B0
:100170006030CB00CE30CC0000308924861EC128F0
:10018000DD20B923A010061FD028B5016322E82284
:10019000A0106030CB00CE30CC0000308924B923D1
:1001A000A018D328A223861ED72824152B26861F05
:1001B000DB2824112B26C328DC280430B500682452
:1001C0003508033C031DE5288529061FEA28B50AE2
:1001D0000130C6251D255330352574303525613055
:1001E000352574303525693035256F3035256E302D
:1001F0003525203035254E303525613035256D309B
:100200003525653035253A303525203035252030E7
:100210003525203035250D3045253508043C031D96
:1002200014294030C80086213508053C031D1B29D0
:100230004130C80086213508063C031D2229423082
:10024000C80086213508073C031D29294330C80012
:1002500086213508083C031D30294430C80086211A
:100260003508093C031D37294530C800862135086B
:100270000A3C031D3E294630C800862135080B3C48
:10028000031D45294730C800862135080C3C031D55
:100290004C294830C800862135080D3C031D5329E0
:1002A0004930C800862135080E3C031D5A294A30C2
:1002B000C800862135080F3C031D61294B30C8005A
:1002C00086213508103C031D68294C30C800862162
:1002D0003508113C031D6F294D30C80086213508B3
:1002E000123C031D76294E30C80086213508133C88
:1002F000031D7D294F30C80086210C304525350867
:10030000143C031D8429E822E028232D3508043CF1
:10031000031D8C293808C9003508053C031D9229A6
:100320003908C9003508063C031D98293A08C90058
:100330003508073C031D9E293B08C9003508083CC9
:10034000031DA4293C08C9003508093C031DAA293E
:100350003D08C90035080A3C031DB0293E08C90004
:1003600035080B3C031DB6293F08C90035080C3C75
:10037000031DBC294008C90035080D3C031DC229D6
:100380004108C90035080E3C031DC8294208C900B0
:1003900035080F3C031DCE294308C9003508103C21
:1003A000031DD4294408C9003508113C031DDA296E
:1003B0004508C9003508123C031DE0294608C9005C
:1003C0003508133C031DE6294708C90048081F25C6
:1003D000861EEB29C90A4908803C031DF1292030FB
:1003E000C900861FF62901304902C90049081F3C8F
:1003F000031DFC297F30C90049083D2548081F25F9
:100400000130C6253508043C031D082A4908B800F8
:100410003508053C031D0E2A4908B9003508063C7D
:10042000031D142A4908BA003508073C031D1A2A7F
:100430004908BB003508083C031D202A4908BC00B8
:100440003508093C031D262A4908BD0035080A3C29
:10045000031D2C2A4908BE0035080B3C031D322A17
:100460004908BF0035080C3C031D382A4908C00064
:1004700035080D3C031D3E2A4908C10035080E3CD5
:10048000031D442A4908C20035080F3C031D4A2AAF
:100490004908C3003508103C031D502A4908C40010
:1004A0003508113C031D562A4908C5003508123C81
:1004B000031D5C2A4908C6003508133C031D622A47
:1004C0004908C70008003508033C031D682A782A3C
:1004D000061F6D2AB50A0130C6253508013C031DEB
:1004E000722A79223508023C031D772AE822632A02
:1004F000232DCB236030CB00CE30CC00203089249C
:1005000024152B261D2553303525653035257430AF
:1005100035252030352554303525583035252030C7
:100520003525861FA72AB70A05303302B3003308E2
:10053000053EB400053034020318A12A013032020E
:10054000B200053034020318A72A6430B307861EB0
:10055000B22AB70A0530B30733085F3C0318B22A42
:10056000B20AB3013208163C031DBD2A3308053C0C
:10057000031DBD2A0130B200B3010130320203185D
:10058000C42A1630B200B3013208563EAE002E081F
:10059000633C0318CE2A0130B000CF2AB0013308E3
:1005A0005F3C0318D42AB3014B233308B1000A304F
:1005B0003702031CE02A0130D4250B30B700E22AB1
:1005C0000130C6256030CB00CE30CC000030892C05
:1005D0000130CA00300806260230CA002E0806265E
:1005E0000330CA00310806260430CA003308062644
:1005F0000530CA00320806260630CA00280806263A
:100600000730CA00290806260830CA00380806261E
:100610000930CA00390806260A30CA003A080626F8
:100620000B30CA003B0806260C30CA003C080626E0
:100630000D30CA003D0806260E30CA003E080626C8
:100640000F30CA003F0806261030CA0040080626B0
:100650001130CA00410806261230CA004208062698
:100660001330CA00430806261430CA004408062680
:100670001530CA00450806261630CA004608062668
:100680001730CA00470806264B23CB230530CD255B
:100690000330B50008003308D3000A30D4006326C5
:1006A000CA004A08AF002E08A6002708CB0026087B
:1006B000CC002D08CD000A307C234B08A7004C0845
:1006C000A6004D08AD00A801A90126082F07A80023
:1006D00027080318013E2D07A9002D08CB00290883
:1006E000CC002808CD0002307C234B08AD004C081C
:1006F000A9004D08A8000800CE004C08CB004D080A
:10070000CC00CD014B08CF004C08D0000830D10000
:10071000CE0C0318902BD10B882BCB01CC010034CD
:1007200003109B2BCE0C031C9B2B5008CC074F08AF
:1007300003184F0FCB07CB0CCC0CCD0CD10B922B4D
:10074000003408006030CB0093244C08CA004A1FD4
:10075000B82B6030CB00CE30CC0024308924CB23A2
:10076000A0141D2520303525203035250130CD251C
:100770000800CB231D25553035254E3035254C300E
:1007800035254F303525433035254B303525203044
:1007900035250130CD2D861AD02B861BD02BB701E5
:1007A0003108553C0319F82B31085F3C0319F82B2D
:1007B00031084B3C0319F82B3108413C0319F82B45
:1007C0003108373C0319F82B31082D3C0319F82B5D
:1007D0003108233C0319F82B3108193C0319F82B75
:1007E00031080F3C0319F82B3108053C031DFC2B85
:1007F0002808013EAA00FE2B2808AA0007301F2562
:100800000430CB003008CC00203066250430CB000B
:100810002E08CC00303078252E3035250430CB0022
:100820003108CC00303078254D30352568303525FD
:100830007A3035256030CB002908CC002A0889247D
:100840000130CD25682C1D25483035254A30352509
:100850004830352527303525533035256F3035253F
:100860006630352574303525203035252630352540
:100870002030352552303525443035255630352544
:1008800056303525203035251B25503035254C3048
:1008900035254C303525203035255430352552301E
:1008A0003525413035254E303525533035254D30F1
:1008B00035254930352554303525543035254530DA
:1008C000352552303525203035250130BF25232DE3
:1008D0001B2538083D2539083D253A083D253B08AC
:1008E0003D253C083D253D083D253E083D253F086A
:1008F0003D2540083D2541083D2542083D2543084A
:100900003D2544083D2545083D2546083D25470829
:100910003D2DCD004B089A244C08B424C5244D0825
:10092000B424C524F72CCC004B08A024A7244D08E0
:10093000CC00C12CCE00042503104E0DB424C52CD0
:10094000CD00042503104D0D013EB424C52CCD006F
:100950000830CE000310CD0DD3244D10201DB12C36
:100960004D14CE0BAA2C0800CF000830D000201167
:10097000CF1FBB2C2015E6240310CF0DD00BB72CB6
:100980000800C324F72C2011E62C1125A2144C26B4
:10099000112522144D2611250518CF2CCC2C1125FC
:1009A00022104D26112D1125A2144C26112522149A
:1009B0004D2611250518DD2CDA2C11252011851C5A
:1009C000E22C2015112522104D26112D1125A210E3
:1009D000201DEB2CA2144C26112522144D26112586
:1009E0000518F32CF02C112522104D26112D112560
:1009F000A2104C26112522104D26112522144D2619
:100A00001125A2144C26112D1125A2144C261125B6
:100A100022144D261125A2104C26112522104D26F8
:100A2000112D0C30F92D24102D2622104D26A41046
:100A30002C26A2104C2EA830452D8030452DCB0001
:100A40004B08803E452D0830452501304525C830EE
:100A5000ED2502304525C830ED25063045250C3002
:100A60004525C830ED2D2108D300D30025162926B1
:100A7000530E0F3951255308512DCB002516292629
:100A80004B0E0F3951254B08512DCC00251229262C
:100A90004C0E0F3951258230ED254C0851258230FE
:100AA000ED2DD400A4152A2654082E26A4112A269A
:100AB000FA30F92D00302E2625122926A4112A26D7
:100AC00000303D2623124926A2114A2ECD004C08A3
:100AD000D0000A30D1005426CE004E08CC004B087E
:100AE000D0004C08D1004D08A0255208CD000800C8
:100AF000CD004C08D0006430D1005426CE004E0802
:100B0000CC004B08D0004C08D3000A30D400632638
:100B1000D2005208D1004D08A0255208CD004C0843
:100B2000D0000A30D1005426CF004F08CC004B082B
:100B3000D0004C08D1004D08A0255208CD00080077
:100B4000D200D108031DAC2DD2080319AB2D5208D9
:100B5000A100500A0620BE2D0A3051020318B62DFE
:100B60005108303EA100500A0620BC2D0A30510227
:100B7000413EA100500A06203030D2000800CA00D1
:100B80004A08CC006430CD00C830DB2DCA004A08CA
:100B9000CC006430CD000A30DB2DCB004B08CC00FC
:100BA0006430CD000130DB2DCA004A08CC000A3089
:100BB000CD000130DB2DCE00FF30CF004D08D1003D
:100BC0004C08D00017304F070318E32DD00BE22D4F
:100BD000D10BE02DCE0BDE2D0800CD004D08CE0050
:100BE000CE08031DF42DF82D0A30F925CE03F02D83
:100BF0000800D500F430D600FC30D7005508560761
:100C0000031C003457070318022E0800CB00831280
:100C100003134B0883169A0083124A0883169B001D
:100C20001C158B138B1355309D00AA309D009C140E
:100C30009C18182E1C118B1783120800CB008312EE
:100C400003134A0883169B001C141A088312CB0056
:100C50000800372E3A2E3A2E3A2E3A2ED500550855
:100C60000F39D6002508F0395604A500372E25087F
:100C700086000800240885000800A60026080F3911
:100C8000A7002308F0392704A3004E2E4E2E4E2E27
:100C90004E2E4E2E512E512E512E512E23086600CF
:100CA0000800220865000800D100D1080319612E50
:100CB0005108500203185D2E612E51085002D000D9
:100CC000582E50080800D400D501D4080319722EFC
:100CD0005408530203186D2E722E54085302D30089
:100CE000D50A682E550808000430A1000800FF3F0F
:100CF000FF3FFF3FFF3FFF3FFF3FFF3FFF3FFF3F04
:100D0000FF3FFF3FFF3FFF3FFF3FFF3FFF3FFF3FF3
:100D1000FF3FFF3FFF3FFF3FFF3FFF3FFF3FFF3FE3
:100D2000FF3FFF3FFF3FFF3FFF3FFF3FFF3FFF3FD3
:02400E00180395
:10420000FF0000006100460046000B00A20007000E
:1042100044006900740020006900730020006500FC
:1042200065006E00200054006500730074002100DA
:10423000FF00FF00FF00FF00FF00FF00FF00FF0086
:10424000FF00FF00FF00FF00FF00FF00FF00FF0076
:10425000FF00FF00FF00FF00FF00FF00FF00FF0066
:10426000FF00FF00FF00FF00FF00FF00FF00FF0056
:10427000FF00FF00FF00FF00FF00FF00FF00FF0046
:10428000FF00FF00FF00FF00FF00FF00FF00FF0036
:10429000FF00FF00FF00FF00FF00FF00FF00FF0026
:1042A000FF00FF00FF00FF00FF00FF00FF00FF0016
:1042B000FF00FF00FF00FF00FF00FF00FF00FF0006
:1042C000FF00FF00FF00FF00FF00FF00FF00FF00F6
:1042D000FF00FF00FF00FF00FF00FF00FF00FF00E6
:1042E000FF00FF00FF00FF00FF00FF00FF00FF00D6
:1042F000FF00FF00FF00FF00FF00FF00FF00FF00C6
:00000001FF
